:020000040000FA
:020000000428D2
:08000800FF30A200FF30A3004D
:100010008B011D2222108422A2108322221182220F
:10002000A2138122FF308522A501A601A701A80104
:10003000A901AA01AB01AC01AD01AE01AF01B00154
:10004000B201B301B401A010B501B601B701C430CB
:100050004A22A016E8212012ED212015F721D121F6
:10006000A01D3328342835282F288101D121A01D37
:100070003A283C283B2836280108B1008101082293
:100080003108503C031820293408013C031D49283D
:10009000B028D121A01D4D284E2852283408013CFB
:1000A000031D53285E282011F7210108A600260809
:1000B000C83C03185D280130B40049288101340888
:1000C000013C0319A8283708093EB8002608380261
:1000D000031881283008BC002F08BD002E08BE0080
:1000E0002D08BF002C08C0000130FC213C08B000E6
:1000F0003D08AF003E08AE003F08AD004008AC0030
:1001000097283008BC002F08BD002E08BE002D081F
:10011000BF002C08C0000030FC213C08B0003D08A6
:10012000AF003E08AE003F08AD004008AC00260816
:10013000B700201126082221D121A01DA028A22825
:10014000A1289C280108A50081012015250822214D
:10015000B20A3208273C0318AF280130B400442803
:100160003408013C031D20292015F72132081B3CCF
:10017000031DF128AD21201EBF282015C028201105
:10018000C221201FC428CD28C528201DCD2820121B
:10019000ED21E02101308D22F0289821A01ED228E7
:1001A000A015D328A011C221201FD728E028D828C5
:1001B000A01DE0282016ED21E02101308D22F0283D
:1001C0008321201FE5282016E6282012C221201FA7
:1001D000EA28EB28F028201EF028E02101308D22AB
:1001E00020296E21201E20293308243C031D2029AC
:1001F00027080C3C031D02292012ED21E0210130CB
:100200008D22202927080D3C031D0C292016ED21E5
:10021000E02101308D222029C221201F1029202910
:1002200011292708493C03191D2927084A3C0319AD
:100230001D292708473C031D2029E02101308D227C
:100240002D282129B900BA01201D2829FF30BA0024
:100250001530390203182F290130B9004029243004
:100260003902031836290230B900402950303902CA
:1002700003183D290330B90040290430B900082291
:100280000330390203186B2935083907BB000230E7
:100290003B02031C64292B08BC002A08BD00290866
:1002A000BE002808BF002708C0003A08FC213C080F
:1002B000AB003D08AA003E08A9003F08A80040087E
:1002C000A700B30AB5016A29A010201D6829A0144F
:1002D0003908B5006D29B501A01008002012AA0840
:1002E000031D8229AB08031D822929080F3C031D29
:1002F00082292808843C031981292808043C031D0D
:100300008229201608002013AF08031D9729B00882
:10031000031D97292E08D23C031D97292D080A3C5E
:10032000031D97292C08883C031D972920170800D6
:10033000A012AF08031DAC29B008031DAC292E087C
:10034000D03C031DAC292D084A3C031DAC292C08C8
:100350000A3C031DAC29A01608002012AF08031D9B
:10036000C129B008031DC1292E08D23C031DC12993
:100370002D08AA3C031DC1292C08953C031DC12949
:1003800020160800B8010330B900861AC829B80A37
:10039000B90BC5292013023038020318D0292017C1
:1003A0000800B9010330BA008619D729B90ABA0B77
:1003B000D429A011023039020318DF29A015080042
:1003C000A012E8210130942201309B22A016E829D6
:1003D000A410A01EEC29A4147C2A2410201EF129AC
:1003E00024147D22A413201AF629A4177A2A241192
:1003F000201DFB2924157B2AC100411C012A03145E
:10040000022A0310C00DBF0DBE0DBD0DBC0D0800AE
:100410000130B200B301A501A601B601B701B401D4
:10042000A701A801A901AA01AB01AC01AD01AE0170
:10043000AF01B001B501A01008008B0120304422AB
:1004400026228030980010309804080006303522AB
:10045000A014A01C302A3B22270804384422342A46
:100460003B222708FB3944220800A500B901993036
:10047000BA002508502AA9019830AA0065222B0845
:10048000A8002808A7000800A500B9019830BA0004
:100490002508502AB800B9018130BA003808502A1E
:1004A000BB00831F552A2015562A2011391C5A2AB1
:1004B00083175B2A83133A0884003B088000201DC1
:1004C000632A8317642A83130800AB00831F6A2AF8
:1004D00020156B2A2011291C6F2A8317702A831379
:1004E0002A0884000008AB00201D782A8317792A87
:1004F000831308007E2A7E2A7E2A7E2A240885000D
:1005000008008A2A8A2A8A2A8A2AA300872A230894
:1005100066000800220865000800B8003808B90025
:10052000FA30BA00C830A22AB8003808B9006430DE
:10053000BA001430A22AB8003808B9006430BA00F2
:100540000530A22ABB00FF30BC003A08BE003908C3
:10055000BD0017303C070318AA2ABD0BA92ABE0B01
:08056000A72ABB0BA52A080025
:02400E00903FE1
:00000001FF
